:020000020000FC
:0400000007C0D3C0A2
:10000C003EC16CC10FED0DBF0FE007BB4424992717
:10001C00C3D2872D8F7E09E009B908E90AB91CD033
:10002C0071E016D373E014D3789468D19BD1FDCFD3
:10003C00C29AC3989860906433D000270BBF46D106
:10004C0080FD03C09298C09802C0929AC09A98D032
:10005C0004E701BB939A0895C298C39A84FF1BD0FE
:10006C0084FD1ED080FFC09880FDC09A82FFC1988D
:10007C0082FDC19A00E001BB02BB0FE081FD0AE0EA
:10008C0005BF00EC0ABF00E483FF0BBF977F84FF22
:10009C009F7B16D1089500E6102E202EA1E6BB27DB
:1000AC00EE2408E0D02E089500E6101619F47CE03A
:1000BC00CFD20895C298121409F4202EC22DDD2738
:1000CC00299183FF13C094FF03C0062F48D013C09F
:1000DC00122F169516951695022F077009F0139589
:1000EC00CF9321961A95E9F739D0CF9194FD03C09F
:1000FC00099138E0000F81FF929881FD929A94FD4E
:10010C0004C010F0939801C0939A94FF8B9A43D03B
:10011C0081FF929A81FD929894FD44D03CD02A950F
:10012C0029F094FDE8CF3A9529F7E0CF8B98939A74
:10013C0080FF929880FD929A2ED083FD07C094FF89
:10014C0003C0062F0CD094FF09D025D019D075E030
:10015C0094FD70E17DD29160C29A0895088109D016
:10016C0012B382FD02C0102B02C00095102312BBEB
:10017C000895005318E0110F0A95E9F7012F08951F
:10018C0002B382FF0C7882FD006702BB82FFC1982C
:10019C0082FDC19A089566246394F1F70895C3987B
:1001AC000F935FB6889483990894FF1CDA9419F422
:1001BC0008E0D02EFD92AD3B10F4E39419F47FE0EF
:1001CC0047D269DF93FD08955FBE0F911895EE201D
:1001DC0099F0092F007249F40D2D083019F411977C
:1001EC00FC90DD24F694D394EA949F7D08E072D0C1
:1001FC0000E270D008E06ED008955523E9F35A95CB
:10020C00AA95F4CF0023C1F30027F0CF1F93EE2063
:10021C0099F1EF93FF930F930D2D083021F0FF0C04
:10022C00DA94E9F7FD92E12DFF27E192E694E6944A
:10023C00E694083009F0E394EE0DEE24EF3B38F031
:10024C007FE006D228DF0F91FF91EF9115C008E0F7
:10025C00D02E12960F9194FF02C0102F07C0EE20E3
:10026C0059F410E3139506950077E1F711931E2EC0
:10027C00FF91EF9193FF9160EE241F9108950F93DE
:10028C005FB600ED02BF00B300770C1551F0C02E25
:10029C0082FD0095007783FD07C0002311F0B6DFC7
:1002AC00C39A5FBE0F911895002321F400270BBF52
:1002BC000B2DF5CFB02E00EC0ABF00E40BBFF1CF35
:1002CC0001E003BF09B7026009BF089509B70D7FAC
:1002DC0009BF08955D9BFECF0CB908950F930FB71E
:1002EC000F930CB10B3718F4013608F0005292FF43
:1002FC00302E94600F910FBF0F91189590FF0895B9
:10030C0093FD04C096FF02C074E0A2D1C22DDD277C
:10031C00299138E01991110F10F401E301C000E3A9
:10032C00D9DF2A9519F03A95B1F7F3CF05E4D2DF6E
:10033C000991D0DF0DE0CEDF0AE0CCDF2C2E9E7FC2
:10034C00F894F89412140FB700FD06C0121431F48F
:10035C0096FD06C0EE2021F49EDE02C093FF916054
:10036C007894089592FF0895032D9B7F0B31E1F152
:10037C00083069F197FD0DC00D3091F00D34B1F0DE
:10038C00023511F1033479F0033521F1033109F40D
:10039C0060C0003358F10B3748F593FDAFC008959A
:1003AC0093FD82CE089577DE7CE052C193FD03C0AD
:1003BC003FDE72E04DC150DE73E04AD196FF0895E6
:1003CC0074E046D170E044C193FFCFC0EEC093FD02
:1003DC00FEDE089572E13CD136D10B3199F1033533
:1003EC0031F00235C9F0F8CF93FD2CD0089572DFAF
:1003FC0070E02ED1442443947A2EC6D0712CC4D0F4
:10040C00722CC2D0112D1056F0E0E0E621F0719064
:10041C00BBD01A95FBCF08955DDF70E019D1442451
:10042C004394BAD0A72DB8D0172CB6D0272C112DA9
:10043C001056F0E0E0E621F0AFD071921A95FBCFA8
:10044C0008958A2DA1E0A10D9F742ADE70E000D1E1
:10045C000895A82E76E0FCD078E011E0F9D0082FB2
:10046C00012311F400E301C001E334DF7395110F94
:10047C001031A1F70DE02EDFE6D00D3011F10B316C
:10048C0001F3033431F481FF02C08D7FE5CF82602C
:10049C00E3CF053431F482FF02C08B7FDDCF846063
:1004AC00DBCF0C3431F483FF02C0877FD5CF88605B
:1004BC00D3CF033509F780FF02C08E7FCDCF81608B
:1004CC00CBCF70E0C5D077E0C3D0BDD00B31C1F23B
:1004DC00033505E531F44424182F1F70712E54D0C8
:1004EC0003E5F8DE70E0B4D093FF04C0A1DD72E048
:1004FC00AFD00895B1DD73E0ABD008950F9395FDA7
:10050C000FC00053023060F497FD02C071E1A0D01F
:10051C009068889400FD089448DE0F91DBDE089506
:10052C000F9195FD07C097FF1FC00534E9F4D2DE8B
:10053C00906208950133C0F00433B0F4CBDE19DEC1
:10054C000F9381D0083021F442DE90620F91089510
:10055C000B3111F477DFFACF0D3099F70F919F77AC
:10056C009F7D54DE70E074D00895092F007439F427
:10057C009064806174E06CD070E06AD004C09F7BA2
:10058C008F7E73E065D00895E199FECF4EBA439407
:10059C007DBAE29AE19A0895E199FECF4EBA43945E
:1005AC00E09A7DB2089570E053D07DE051D055278C
:1005BC004AD00B3111F446DF0895083011F41DDEDA
:1005CC00F7CF0D3051F0003398F30A3388F7539579
:1005DC0081DE00530D93533059F7552349F32E9177
:1005EC005A9561F00E9129D0200F5A9539F00E9141
:1005FC000330C8F622D021D0200FA8F2222399F282
:10060C0070E026D07EE024D01ED00B31A1F2013355
:10061C00D8F30433C8F7602F5DDE15D0083011F421
:10062C00F1DDF2CF0D30C9F770E012D09061212CC2
:10063C0048DD062FEBDD9F7E0895000F402F000F45
:10064C00000F040F089592FFFECF032D9B7F08959A
:10065C000F93ECE8F6E0972E990C8824E90DF81D21
:10066C00C895802C3196C895902CE82DF92DC895FD
:10067C003196002019F0002D2DDEF9CF0F91089541
:10068C000107B206E406F40604070E071607340742
:10069C004C0758076607740782079207A807B80724
:1006AC00D407DC07E407332D776972652D62757307
:1006BC002D696E746572666163652056312E31202A
:1006CC0028632920557765204B65727769656E2004
:1006DC00323030330D0A00006D6F64653A206D6165
:1006EC00737465720D0A00006D6F64653A206D6F4E
:1006FC006E69746F720D0A007265636F72643A20D2
:10070C00000073656E643A20000073657475703A6E
:10071C002028746F67676C65206D697420532C43B7
:10072C002C452C4C290D0A0073746F72652F757350
:10073C00652073657475702028532F55293A200055
:10074C00436C6F636B5345543D2000002C20436C6D
:10075C006F636B504F4C3D2000002C20456E616246
:10076C006C65504F4C3D20002C20456E61626C65D1
:10077C004C454E3D200062756666657220656D7055
:10078C007479210D0A00626974206E756D62657250
:10079C002028312D323535293A200000656E6162F2
:1007AC006C652028312D33293A2000004552524FD8
:1007BC00523A20627566666572206F766572666C59
:1007CC006F7720210D0A0000726561643A200000E9
:1007DC00696E7075743A200073746F72652F726550
:1007EC0063616C6C206275666665722028532F52AB
:0407FC00293A200076
:00000001FF
